:100000000C942E020C9472020C9472020C947202E4
:100010000C9472020C9472020C9472020C94720290
:100020000C9472020C9472020C94280C0C94FA0C2E
:100030000C94FD1A0C9472020C9472020C947202CD
:100040000C9472020C9472020C9472020C94720260
:100050000C9472020C946A1B0C9472020C9472023F
:100060000C9472020C9472020C9472020C94720240
:100070000C9472020C9472020C9472020C94720230
:100080000C9472020C9472020C9472020C94720220
:100090000C9472020C9472020C9472020C94720210
:1000A0000C9472020C9472020C9472020000F1A47F
:1000B000F1A3018C028C048C2B0014001A000800A0
:1000C000150017001C0018000C00120013002A0075
:1000D000290004001600070009000A000B000D00AB
:1000E0000E000F0033003400E1001D001B0006006D
:1000F00019000500110010003600370038002800F4
:100100000030E000E200E30002202C002C0001207F
:100110005000510052004F002B0014001A0009003B
:1001200013000A000D000F0018001C0033002A0005
:100130002900040015001600170007000B0011002D
:1001400008000C0012003400E1001D001B00060036
:10015000190005000E001000360037003800280096
:100160000030E000E200E30002202C002C0001201F
:100170005000510052004F002B0034003600370071
:1001800013001C0009000A00060015000F002A00D9
:10019000290004001200080018000C0007000B00E2
:1001A0001700110016003800E100330014000D00A4
:1001B0000E001B00050010001A0019001D00280089
:1001C0000030E000E200E30002202C002C000120BF
:1001D0005000510052004F0035021E021F02200243
:1001E00021022202230224022502260227022A00DB
:1001F00001003A003B003C003D003E003F002D0264
:100200002E022F0230023102010040004100420064
:100210004300440045000320042005200050010055
:1002200001000100010001000220010001000100A5
:10023000AB00AA00A900AE0035001E001F00200080
:1002400021002200230024002500260027002A0088
:1002500001003A003B003C003D003E003F002D0005
:100260002E002F003000310001004000410042000C
:1002700043004400450003200420052000500100F5
:100280000100010001000100010001000100012046
:10029000AB00AA00A900AE00280354006800650066
:1002A000200050006C0061006E0063006B002000B5
:1002B0004B006500790062006F006100720064000D
:1002C00000002C034F007200740068006F006C0087
:1002D00069006E0065006100720020004B0065003F
:1002E000790062006F00610072006400730000001A
:1002F0000403090409027400040100A03209040087
:10030000000103010100092111010001223F000742
:1003100005810308000A0904010001030102000924
:100320002111010001224D000705820308000A097E
:10033000040200010300000009211101000122361E
:10034000000705830308000A0904030002030000F4
:10035000000921110100012220000705840320006B
:10036000010705040320000112011001000000082C
:10037000EDFE60600100010200010631FF0974A179
:10038000010975150025FF9520750881020976156C
:100390000025FF952075089102C005010980A10183
:1003A000850216010026B7001A01002AB700751051
:1003B00095018100C0050C0901A10185031601000A
:1003C000269C021A01002A9C02751095018100C02A
:1003D00005010902A1010901A10005091901290569
:1003E00015002501950575018102950175038101AF
:1003F0000501093009311581257F950275088106AF
:1004000009381581257F950175088106050C0A3884
:10041000021581257F950175088106C0C005010977
:1004200006A101050719E029E715002501950875C2
:1004300001810295017508810105081901290595B9
:1004400005750191029501750391010507190029B0
:10045000FF150025FF950675088100C011241FBEF9
:10046000CFEFDAE0DEBFCDBF04B603FE24C080913B
:10047000EA019091EB01A091EC01B091ED01873080
:10048000904BA740B04BB9F41092EA011092EB01E7
:100490001092EC011092ED0114BE84B7877F84BFE7
:1004A00088E10FB6F89480936000109260000FBE50
:1004B000E0E0F8E3099511E0A0E0B1E0E6ECF7E454
:1004C00002C005900D92A235B107D9F711E0A2E55F
:1004D000B1E001C01D92AA3EB107E1F70E947C097C
:1004E0000C94E1230C9400000895089561110DC04F
:1004F000FC018281882331F085EE0E940D100E945C
:10050000262203C085EE0E94D51080E090E0089579
:100510008B3B910568F4883A910530F5853A910551
:10052000C0F48430910598F4019709F06FC071C050
:10053000803E910508F46AC0883E910540F09C0118
:10054000205F31092031310508F060C05CC09C019A
:10055000A1C0853A910509F45FC0863A910509F476
:100560005EC023E830E496C0883A910509F45AC089
:10057000893A910509F459C08A3A910509F458C09D
:100580008B3A910509F457C08C3A910509F456C08D
:100590008D3A910509F455C0803B910509F454C08A
:1005A0008E3A910509F453C08F3A910509F452C06F
:1005B000813B910509F451C0823B910509F450C07B
:1005C000833B910509F44FC0843B910509F44EC06B
:1005D000853B910509F44DC0863B910509F44CC05B
:1005E000873B910509F44BC0883B910509F44AC04B
:1005F000893B910509F449C08A3B910509F048C03F
:100600002AE236E447C09C01306544C020E030E077
:1006100041C021E030E03EC021E830E43BC022E8A8
:1006200030E438C022EE34E435C029EE34E432C080
:100630002AEE34E42FC025EB34E42CC026EB34E45E
:1006400029C027EB34E426C02CEC34E423C02DEC85
:1006500034E420C023E835E41DC02AE835E41AC09C
:1006600022E935E417C024E935E414C021E236E478
:1006700011C023E236E40EC024E236E40BC025E2CA
:1006800036E408C026E236E405C027E236E402C0BC
:1006900020E034E4C901089508959CE0799FF001B9
:1006A000112490E3899FE00DF11D1124E60FF11D47
:1006B000EE0FFF1FE854FF4F25913491C9010895B3
:1006C000880F991F845D9040FC0125913491C901E8
:1006D0000895880F991F84559F4FFC0125913491EF
:1006E000C90108950E944D039C013A9521153F418F
:1006F00008F4DFC09C0130522115304120F49F7076
:100700000E94690308959C0130532115304118F46B
:100710009927906C08959C0130542031310520F4C4
:100720008F709927946D0895803120E4920719F411
:1007300080E091ED0895813140E4940719F480E060
:1007400090ED0895823120E4920719F480E092ED53
:100750000895833140E4940719F480E093ED0895FF
:10076000811520E5920711F40C948F1B813040E530
:10077000940731F48091C70181608093C701089587
:100780009C0130562115304108F402C097FF02C089
:10079000906F0895803E9105E0F4803C910568F5E6
:1007A0008133910509F474C048F48932910509F444
:1007B0006AC08A32910509F07AC074C08933910504
:1007C000F9F082389105E1F08533910509F06FC0A9
:1007D00050C0833E9105A9F140F4803E9105C9F0D7
:1007E000823E910509F063C01BC0863E910571F100
:1007F000873E910509F05BC037C00E9460030895F1
:100800002091DA0120FD02C021FF51C080EE90E06E
:100810004EC08091DA0180FFF9CF89E390E047C0B4
:100820008091DA0182FF0AC08091DA0184FF03C05F
:1008300080E090E03CC083EE90E039C082EE90E032
:1008400036C08091DA0182FFEFCFF8CF8091DA01D4
:1008500083FF07C08091DA0184FDEACF87EE90E044
:1008600026C086EE90E023C08091DA0183FFF2CFAC
:10087000F8CF8091DA0185FF03C089E290E017C0CC
:1008800085E390E014C08091DA0185FDF9CFF5CFC2
:100890008091DA0186FF03C08AE290E008C081E31C
:1008A00090E005C08091DA0186FDF9CFF5CF0E9476
:1008B000880208955F926F927F928F929F92AF927B
:1008C000BF92CF92DF92EF92FF920F931F93CF933D
:1008D000DF93CDB7DEB728970FB6F894DEBF0FBE13
:1008E000CDBF9E012F5F3F4F4E0189E0880E911CC6
:1008F00060E070E000E010E0E12CF12CC12CD12C84
:10090000A12CB12C88E0782E622E532E41E050E0CD
:10091000E4E1F1E0A62DB52D872D01900D928A9589
:10092000E1F7F901819191919F01FC01E07FFF279F
:10093000E032F10559F48F709927FA0102C0EE0FE9
:10094000FF1F8A95E2F7AE2ABF2A37C0E033F105D0
:1009500059F48F709927FA0102C0EE0FFF1F8A9594
:10096000E2F7CE2ADF2A29C0E034F10559F48F706E
:100970009927FA0102C0EE0FFF1F8A95E2F7EE2ACF
:10098000FF2A1BC0E035F10559F48F709927FA0151
:1009900002C0EE0FFF1F8A95E2F70E2B1F2B0DC032
:1009A000E036F10551F48F709927FA0102C0EE0F7D
:1009B000FF1F8A95E2F76E2B7F2B2815390509F06A
:1009C000A7CF94B18A2D8095892384B985B18A29CE
:1009D00085B997B18C2D8095892387B988B18C29E9
:1009E00088B99AB18E2D809589238AB98BB18E29C9
:1009F0008BB99DB1802F809589238DB98EB1802BC5
:100A00008EB990B3862F8095892380BB81B3862BC6
:100A100081BB28960FB6F894DEBF0FBECDBFDF9125
:100A2000CF911F910F91FF90EF90DF90CF90BF90EB
:100A3000AF909F908F907F906F905F9008955F929E
:100A40006F927F928F929F92AF92BF92CF92DF92DE
:100A5000EF92FF920F931F93CF93DF93CDB7DEB743
:100A600068970FB6F894DEBF0FBECDBF85B780681C
:100A700085BF85B7806885BF6E9A769A0E945A04B2
:100A80009E012F5F3F4F4E0189E1880E911C60E06F
:100A900070E000E010E0E12CF12CC12CD12CA12C55
:100AA000B12C98E1792E622E532E41E050E0ECE11A
:100AB000F1E0A62DB52D872D01900D928A95E1F7D5
:100AC000F901819191919F01FC01E07FFF27E032C4
:100AD000F10559F48F709927FA0102C0EE0FFF1F3C
:100AE0008A95E2F7AE2ABF2A37C0E033F10559F400
:100AF0008F709927FA0102C0EE0FFF1F8A95E2F767
:100B0000CE2ADF2A29C0E034F10559F48F709927E5
:100B1000FA0102C0EE0FFF1F8A95E2F7EE2AFF2AC4
:100B20001BC0E035F10559F48F709927FA0102C016
:100B3000EE0FFF1F8A95E2F70E2B1F2B0DC0E0363C
:100B4000F10551F48F709927FA0102C0EE0FFF1FD3
:100B50008A95E2F76E2B7F2B2815390509F0A7CF70
:100B600094B18A2D8095892384B985B18A2985B964
:100B700097B18C2D8095892387B988B18C2988B944
:100B80009AB18E2D809589238AB98BB18E298BB924
:100B90009DB1802F809589238DB98EB1802B8EB920
:100BA00090B3862F8095892380BB81B3862B81BB30
:100BB000109253011092520110925B0110925A014F
:100BC000109255011092540110925D0110925C0137
:100BD000109257011092560110925F0110925E011F
:100BE0001092590110925801109261011092600107
:100BF00068960FB6F894DEBF0FBECDBFDF91CF91E0
:100C00001F910F91FF90EF90DF90CF90BF90AF902A
:100C10009F908F907F906F905F9008955F926F92FA
:100C20007F928F929F92AF92BF92CF92DF92EF927C
:100C3000FF920F931F93CF93DF93CDB7DEB7A097AB
:100C40000FB6F894DEBF0FBECDBF7E0149E1E40EC2
:100C5000F11C2AE5C22E21E0D22E5E0151E2A50E42
:100C6000B11C38E0532E470101E010E048E1642E4A
:100C700055E0752EE4E1F1E0D401852D01900D924F
:100C80008A95E1F7F701819191917F019C01207F85
:100C900033272032310589F424B18F709927A801B8
:100CA00002C0440F551F8A95E2F7CA01242B24B9CC
:100CB00095B18095892385B94FC02033310589F4DA
:100CC00027B18F709927F80102C0EE0FFF1F8A9598
:100CD000E2F7CF012E2B27B998B18095892388B9E7
:100CE0003BC02034310589F42AB18F709927A801BF
:100CF00002C0440F551F8A95E2F7CA01242B2AB976
:100D00009BB1809589238BB927C02035310589F4A3
:100D10002DB18F709927F80102C0EE0FFF1F8A9541
:100D2000E2F7CF012E2B2DB99EB1809589238EB984
:100D300013C02036310581F420B38F709927A801A4
:100D400002C0440F551F8A95E2F7CA01242B20BB2D
:100D500091B38095892381BB50EA5A95F1F7BE0182
:100D60006F5F7F4F80E090E020E030E0ECE1F1E069
:100D7000DE011196462D01900D924A95E1F7FB0197
:100D800041915191BF01FA01E07FFF27E032F10567
:100D900011F4E3B113C0E033F10511F4E6B10EC074
:100DA000E034F10511F4E9B109C0E035F10511F4C1
:100DB000ECB104C0E036F105B9F4EFB1F0E04F70EA
:100DC000552702C0F595E7954A95E2F7E0FD08C082
:100DD000A801022E02C0440F551F0A94E2F702C078
:100DE00040E050E0842B952B2F5F3F4F2C30310596
:100DF00009F0BCCFF601208131812817390721F095
:100E000091838083709200010E945A04F2E0CF0E19
:100E1000D11CEA14FB0409F02DCF80910001882336
:100E200061F1815080930001811121C080915A01AC
:100E300090915B01909353018093520180915C01EA
:100E400090915D01909355018093540180915E01D2
:100E500090915F01909357018093560180916001BA
:100E600090916101909359018093580106C08FE9D8
:100E70009FE00197F1F700C0000081E0A0960FB657
:100E8000F894DEBF0FBECDBFDF91CF911F910F91C0
:100E9000FF90EF90DF90CF90BF90AF909F908F909A
:100EA0007F906F905F900895E82FF0E0EE0FFF1FA6
:100EB000EE5AFE4F80819181089508950895811121
:100EC0000BC080918000877F8093800010928D00FE
:100ED00010928C002F9808952F98833041F48091C0
:100EE00080008860809380008FEF9FEF12C0909108
:100EF000800098609093800023E030E0281B310947
:100F0000220F331F8FEF9FEF02C0969587952A958A
:100F1000E2F790938D0080938C00089580916B018F
:100F20000895CF93DF9300D01F92CDB7DEB7209105
:100F3000E001243021F523E029839B838A832093D9
:100F4000E9008FEF06C095ED9A95F1F70000882330
:100F500029F09091E800815095FFF5CF8091E8004D
:100F600085FF0DC040E050E063E070E0CE010196E7
:100F70000E94150A8091E8008E778093E8000F9018
:100F80000F900F90DF91CF910895CF93DF9300D012
:100F90001F92CDB7DEB72091E001243029F522E081
:100FA00029839B838A8383E08093E9008FEF06C0C7
:100FB00095ED9A95F1F70000882329F09091E800CB
:100FC000815095FFF5CF8091E80085FF0DC040E08E
:100FD00050E063E070E0CE0101960E94150A809116
:100FE000E8008E778093E8000F900F900F90DF91CC
:100FF000CF9108952091E0012430F9F422E020936C
:10100000E9002FEF06C035ED3A95F1F700002223F5
:1010100029F03091E800215035FFF5CF2091E8000C
:1010200025FF0BC040E050E065E070E00E94150A2B
:101030008091E8008E778093E8000895CF93DF9346
:10104000EC018091E001843041F581E08093E9007A
:101050008FEF06C095ED9A95F1F70000882329F0EF
:101060009091E800815095FFF5CF8091E80085FFD1
:1010700014C040E050E068E070E0CE010E94150A24
:101080008091E8008E778093E80088E0FE01A3E677
:10109000B1E001900D928A95E1F7DF91CF9108952B
:1010A0008091DF01811109C00E94AD0B0E940A0CE2
:1010B0008091E20084608093E20008951092DF0145
:1010C000089508950C9475020C94F91A8091E0012A
:1010D000843049F58091E9008F709091EC0090FF89
:1010E00002C090E801C090E0982B84E08093E90072
:1010F0008091EB0080FF14C08091EE0087FD03C05B
:101100000FC01092F1008091E80085FDFACF809128
:10111000E80080FF05C08091E8008E778093E800AA
:101120009F709093E900089542E061EC81E00E9495
:10113000230B42E061EC82E00E94230B42E061EC71
:1011400083E00E94230B46E261EC84E00C94230BC5
:101150008091E201833009F454C030F4813071F0A1
:10116000823009F0AAC091C08A3009F47EC08B3069
:1011700009F45FC0893009F0A0C020C08091E1016E
:10118000813A09F09AC08091E800877F8093E80057
:101190008091E5019091E601892B21F060E080E0EB
:1011A00090E003C068E083E691E070E00E94640A8A
:1011B0008091E8008B778093E80008958091E101A9
:1011C000813209F07AC08091E5019091E601892B86
:1011D00009F073C08091E800877F8093E80005C024
:1011E0008091E001882309F468C08091E80082FFC3
:1011F000F7CF8091F10080936B018091E8008B77AD
:1012000058C08091E101813A09F057C08091E50111
:101210009091E601892B09F050C08091E800877F0A
:101220008093E8008091E80080FFFCCF80910B0163
:101230003BC08091E101813209F03FC08091E5011E
:101240009091E601892BC9F58091E800877F809312
:10125000E8000E945A0B9091E30181E0911101C0D6
:1012600080E080930B010C94FC148091E1018132A9
:1012700021F58091E800877F8093E8000E945A0B57
:101280008091E4018093620108958091E101813AA7
:10129000A1F48091E800877F8093E8008091E800C6
:1012A00080FFFCCF809162018093F1008091E80083
:1012B0008E778093E8000C945A0B089584B7877F4B
:1012C00084BF88E10FB6F8948093600010926000AC
:1012D0000FBE90E080E80FB6F89480936100909381
:1012E00061000FBE0E94AD0B0E940A0CE2EEF0E01E
:1012F00080818460808308950E945E0978940E94B2
:10130000A70E0E941C0F81E091E00E94C40E0BC04A
:101310000E94BE1A8091DE01882329F00E94E41AFF
:1013200081110E94FF098091E001853089F30E94BC
:10133000260FF9CF292F332723303105B1F04CF494
:101340002130310509F44DC02230310509F04EC07D
:1013500007C02132310541F12232310591F146C0F9
:10136000E4E7F0E084EF92E045C0992781309105F1
:1013700069F08230910589F0892B09F037C0E0EFE0
:10138000F2E0E491F0E080EF92E034C0E2ECF2E0D1
:10139000E491F0E082EC92E02DC0E8E9F2E0E49123
:1013A000F0E088E992E026C0643000F5E62FF0E036
:1013B000EE0FFF1FEC5CFE4F80819181E9E0F0E0D1
:1013C00019C0643098F4E62FF0E0DF01AA0FBB1FCC
:1013D000A45CBE4F8D919C91EC5BFE4FE081F0E0F0
:1013E00009C0E2E1F0E088E693E004C0E0E0F0E06C
:1013F00080E090E0DA018D939C93CF01089580E125
:1014000089BD82E189BD09B400FEFDCF8091D8007D
:101410008F7D8093D8008091E00082608093E0000F
:101420008091E00081FDFCCF0895BF92CF92DF92C2
:10143000EF92FF920F931F93CF93DF937C018B0169
:10144000EA010E947B0BB82E811133C0209731F046
:1014500028813981021B130BE20EF31EC12CD12C03
:1014600023C08091E80085FD15C08091E8008E774B
:101470008093E800209749F0888199818C0D9D1D0B
:101480009983888325E0B22E14C00E947B0B8823A9
:1014900059F00EC0F70181917F018093F100015056
:1014A0001109FFEFCF1ADF0A01151105D1F601C0AE
:1014B000B82E8B2DDF91CF911F910F91FF90EF9060
:1014C000DF90CF90BF9008954091E7015091E801DF
:1014D0004617570748F06115710539F44091E80047
:1014E0004E774093E80001C0BA01FC0140E033C0F0
:1014F0008091E001882309F442C0853009F441C09D
:101500008091E80083FD39C08091E80082FD2FC002
:101510008091E80080FF1FC09091F3008091F2005D
:10152000392F20E0A901482BCA0106C04191409300
:10153000F1006150710901966115710519F088304B
:101540009105A0F341E0089709F040E08091E800A0
:101550008E778093E8006115710551F64111C8CF6F
:1015600006C08091E001882351F0853051F08091D0
:10157000E80082FFF6CF80E0089581E0089582E0E0
:10158000089583E008954091E7015091E8014617DE
:10159000570748F06115710539F44091E8004E771E
:1015A0004093E80001C0BA01FC0140E034C08091E2
:1015B000E001882309F443C0853009F442C08091DA
:1015C000E80083FD3AC08091E80082FD30C0809140
:1015D000E80080FF20C09091F3008091F200392F45
:1015E00020E0A901482BCA0107C044914093F100B3
:1015F00031966150710901966115710519F08830B5
:10160000910598F341E0089709F040E08091E800E7
:101610008E778093E8006115710549F64111C7CFB7
:1016200006C08091E001882351F0853051F080910F
:10163000E80082FFF6CF80E0089581E0089582E01F
:10164000089583E00895982F2CC09093E90098178F
:1016500039F07091EC002091ED005091F00003C042
:10166000242F762F50E021FD02C09F5F1AC03091D9
:10167000EB003E7F3093EB003091ED003D7F3093E7
:10168000ED003091EB0031603093EB007093EC0093
:101690002093ED005093F0002091EE0027FDE5CF60
:1016A00007C0973090F28F708093E90081E0089531
:1016B00080E008958091E10187FD05C08091E800F8
:1016C00080FF0EC012C08091E80082FD05C08091AD
:1016D000E0018111F8CF08958091E8008B7708C070
:1016E0008091E0018111EACF08958091E8008E7722
:1016F0008093E80008958091E4009091E50045E62C
:101700002091EC0020FD1FC023C02091E001222386
:1017100091F0253091F02091EB0025FD10C0209133
:10172000E4003091E5002817390751F34150C90111
:1017300039F784E0089582E0089583E0089581E018
:10174000089580E008952091E80020FFDECFF9CFD2
:101750002091E80022FFD9CFF4CF0E941B0C0E94F9
:10176000230CE0EEF0E0808181608083E8EDF0E022
:1017700080818F77808319BCA7EDB0E08C918E7F3C
:101780008C9380818F7E80831092DF0108950F9368
:101790001F93CF93DF930E941B0C0E94230CC8ED74
:1017A000D0E088818F77888388818068888388816A
:1017B0008F7D888319BC1092E0011092DC01109299
:1017C000DE011092DD0100EE10E0F80180818B7FD8
:1017D000808388818160888342E060E080E00E94AD
:1017E000230BE1EEF0E080818E7F8083E2EEF0E07B
:1017F000808181608083808188608083F80180811E
:101800008E7F8083888180618883DF91CF911F9153
:101810000F910895E8EDF0E080818F7E8083E7ED01
:10182000F0E080818160808384E082BF81E08093EA
:10183000DF010C94C70BE8EDF0E080818E7F8083A0
:101840001092E20008951092DA001092E1000895DB
:101850001F920F920FB60F9211242F933F934F9325
:101860005F936F937F938F939F93AF93BF93EF9308
:10187000FF938091E10082FF0BC08091E20082FF24
:1018800007C08091E1008B7F8093E1000E94660891
:101890008091DA0080FF1FC08091D80080FF1BC0BC
:1018A0008091DA008E7F8093DA008091D90080FFEA
:1018B0000DC080E189BD82E189BD09B400FEFDCF84
:1018C00081E08093E0010E94500805C019BC10928D
:1018D000E0010E945E088091E10080FF19C08091C4
:1018E000E20080FF15C08091E2008E7F8093E200CD
:1018F0008091E20080618093E2008091D800806254
:101900008093D80019BC85E08093E0010E946208B2
:101910008091E10084FF30C08091E20084FF2CC000
:1019200080E189BD82E189BD09B400FEFDCF8091CF
:10193000D8008F7D8093D8008091E1008F7E8093C6
:10194000E1008091E2008F7E8093E2008091E200CE
:1019500081608093E2008091DC01882311F084E0B3
:1019600007C08091E30087FF02C083E001C081E0EF
:101970008093E0010E9464088091E10083FF29C008
:101980008091E20083FF25C08091E100877F8093F2
:10199000E10082E08093E0011092DC018091E1009F
:1019A0008E7F8093E1008091E2008E7F8093E20041
:1019B0008091E20080618093E20042E060E080E09C
:1019C0000E94230B8091F00088608093F0000E94B9
:1019D0006108FF91EF91BF91AF919F918F917F919E
:1019E0006F915F914F913F912F910F900FBE0F908C
:1019F0001F9018951F920F920FB60F9211242F93DC
:101A00003F934F935F936F937F938F939F93AF9386
:101A1000BF93CF93EF93FF938091E9008F709091E4
:101A2000EC0090FF02C090E801C090E0C92FC82BE5
:101A30001092E9008091F000877F8093F000789405
:101A40000E943E0D1092E9008091F0008860809322
:101A5000F000CF70C093E900FF91EF91CF91BF915B
:101A6000AF919F918F917F916F915F914F913F9136
:101A70002F910F900FBE0F901F9018951F93CF932B
:101A8000DF93CDB7DEB7AC970FB6F894DEBF0FBECD
:101A9000CDBFE1EEF1E08091F100819321E0E93EDC
:101AA000F207C9F70E94A8088091E80083FF37C1B8
:101AB0008091E1019091E201953009F488C038F4F9
:101AC0009130B1F170F0933009F029C131C09830F4
:101AD00009F4F8C0993009F404C1963009F01FC127
:101AE0009DC0803821F0823809F019C108C080916A
:101AF000DD019091DE01992389F082600FC0809111
:101B0000E5019091E6018F7099278093E90080911B
:101B1000EB0085FB882780F91092E9009091E8009E
:101B2000977F9093E8008093F1001092F100D5C068
:101B3000882319F0823009F0F2C08F7121F08230D1
:101B400009F0EDC00BC08091E301813009F0E7C0DE
:101B5000933009F080E08093DE012FC08091E30193
:101B600081112BC08091E5019091E6018F7099273A
:101B7000009709F4D4C08093E9002091EB0020FF86
:101B80001CC02091E201233021F48091EB0080629F
:101B900012C09091EB0090619093EB0021E030E057
:101BA00001C0220F8A95EAF72093EA001092EA001A
:101BB0008091EB0088608093EB001092E9008091A7
:101BC000E800877F8093E8000E945A0BA8C081112B
:101BD000A6C08091E3019091E4018F779927182F97
:101BE0009091E3009078982B9093E3008091E80027
:101BF000877F8093E8000E945A0B8091E80080FF65
:101C0000FCCF8091E30080688093E300112311F002
:101C100083E001C082E08093E00181C0805882307F
:101C200008F07DC08091E3019091E4018C3D23E0B8
:101C3000920779F583E08A838AE289834FB7F89423
:101C4000DE01139620E03EE051E2E32FF0E05093F6
:101C50005700E49120FF03C0E295EF703F5FEF7003
:101C60008E2F90E0EA3010F0C79601C0C0968D9399
:101C70009D932F5F243149F74FBF8091E800877F04
:101C80008093E8006AE270E0CE0101960E94640A47
:101C900013C0AE01455D5F4F6091E5010E949A0956
:101CA0000097E9F12091E800277F2093E800BC012C
:101CB0008BA59CA50E94C30A8091E8008B77809336
:101CC000E8002DC0803859F58091E800877F809327
:101CD000E8008091DC018093F1008091E8008E772C
:101CE00071CF81111CC09091E3019230C0F48091BA
:101CF000E800877F8093E8009093DC010E945A0BF4
:101D00008091DC01811104C08091E30087FF02C053
:101D100084E001C081E08093E0010E9494088091FA
:101D2000E80083FF0AC08091E800877F8093E80085
:101D30008091EB0080628093EB00AC960FB6F89434
:101D4000DEBF0FBECDBFDF91CF911F910895CF931E
:101D50008091E0018823B1F08091E9008F7090912B
:101D6000EC0090FF02C090E801C090E0C92FC82BA2
:101D70001092E9008091E80083FD0E943E0DCF7033
:101D8000C093E900CF91089590936E0180936D0107
:101D9000089580916D0190916E010895E0916D011B
:101DA000F0916E01309721F00190F081E02D0994BF
:101DB00080E00895E0916D01F0916E01309721F07F
:101DC0000280F381E02D09940895E0916D01F09176
:101DD0006E01309721F00480F581E02D099408957B
:101DE00020916F01309170018217930771F09093E9
:101DF000700180936F01E0916D01F0916E01309759
:101E000021F00680F781E02D099408952091710159
:101E1000309172018217930771F090937201809351
:101E20007101E0916D01F0916E01309721F0008415
:101E3000F185E02D099408950E94261B0E941F053C
:101E40000E94FA1B0C94CF210C945E075F926F9254
:101E50007F928F929F92AF92BF92CF92DF92EF923A
:101E6000FF920F931F93CF93DF93CDB7DEB72A97DF
:101E70000FB6F894DEBF0FBECDBF0E940E0693E7EB
:101E8000C92E91E0D92E00E010E0AA24A394B12C31
:101E9000502E802F0E9454073C01F601E190F190F2
:101EA0006F01E826F926E114F10431F40F5F1F4FAA
:101EB0000430110569F73AC08091C70181FD0E9485
:101EC0005D0720E030E04501022E02C0880C991C1D
:101ED0000A94E2F7C4018E219F21892B09F12E83F8
:101EE0005F826820792081E0672809F480E0888794
:101EF0000E942F1B8160782F9A8789874E815F818E
:101F000068858A850E94DF0FF801EE0FFF1FED58EC
:101F1000FE4F80819181882599259183808316C009
:101F20002F5F3F4F2C30310571F6C0CF8FEF898383
:101F30008A831B820E942F1B8160782F9D838C8354
:101F400049815A816B818D810E94DF0F0E94E71EBB
:101F500010917B010E94CE0E1817D9F00E94CE0E70
:101F600080937B012A960FB6F894DEBF0FBECDBFDB
:101F7000DF91CF911F910F91FF90EF90DF90CF9065
:101F8000BF90AF909F908F907F906F905F900C94D8
:101F9000240F2A960FB6F894DEBF0FBECDBFDF9197
:101FA000CF911F910F91FF90EF90DF90CF90BF9056
:101FB000AF909F908F907F906F905F900895CF9398
:101FC000DF93CDB7DEB72B970FB6F894DEBF0FBE09
:101FD000CDBF4F83588769877A878B87DE0111963B
:101FE00086E0FD0111928A95E9F785E0FE013796BA
:101FF00001900D928A95E1F749815A816B817C812C
:102000008D819E810E94B7172B960FB6F894DEBF84
:102010000FBECDBFDF91CF910895CF93C82F8823F6
:1020200009F4C1C0823859F40E94CE0E81FDBBC0B4
:1020300089E30E941C1A0E94981A89E30CC0833815
:1020400079F40E94CE0E80FDAEC083E50E941C1A7A
:102050000E94981A83E50E943E1ACF910C94981A18
:10206000843859F40E94CE0E82FD9DC087E40E9400
:102070001C1A0E94981A87E4EECF8450813A48F4E3
:102080008C2F0E94372181118EC08C2F0E941C1A28
:10209000E4CF8C2F805E883050F4C77081E090E0F0
:1020A00001C0880FCA95EAF70E945F1AD6CF8C2F1D
:1020B000855A833078F4C53A29F0C63A31F482E87B
:1020C00090E005C081E890E002C083E890E0CF9105
:1020D0000C94F00E8C2F885A833108F064C0C83AF3
:1020E00039F1C93A41F1CA3A49F1CB3A51F1CC3A06
:1020F00059F1CD3A61F1C03B69F1CE3A71F1CF3A75
:1021000079F1C13B81F1C23B89F1C33B91F1C43B01
:1021100099F1C53BA1F1C63BA9F1C73BB1F1C83B61
:10212000B9F1C93BC1F1CA3BC9F58AE292E038C0B6
:1021300082EE90E035C089EE90E032C08AEE90E009
:102140002FC085EB90E02CC086EB90E029C087EB98
:1021500090E026C08CEC90E023C08DEC90E020C095
:1021600083E891E01DC08AE891E01AC082E991E01D
:1021700017C084E991E014C081E292E011C083E2CB
:1021800092E00EC084E292E00BC085E292E008C0CB
:1021900086E292E005C087E292E002C080E090E033
:1021A000CF910C94060FCF910895882309F44DC068
:1021B000823859F40E94CE0E81FF47C089E30E9405
:1021C0001C1A0E94981A89E30CC0833871F40E948B
:1021D000CE0E80FF3AC083E50E941C1A0E94981A16
:1021E00083E50E943E1A0C94981A843859F40E9490
:1021F000CE0E82FF2AC087E40E941C1A0E94981A01
:1022000087E4EFCF982F9450913A08F4EACF982FB3
:10221000905E983058F4282F277081E090E001C03C
:10222000880F2A95EAF70E94651ADDCF982F955AF4
:10223000933020F480E090E00C94F00E885A8331C3
:1022400020F480E090E00C94060F0895882321F09C
:102250000E945F1A0C94981A0895882321F00E9416
:10226000651A0C94981A0895BF92CF92DF92EF925C
:10227000FF920F931F93CF93DF93CDB7DEB72797CE
:102280000FB6F894DEBF0FBECDBF8C0185E0F8011C
:10229000DE01119601900D928A95E1F7F8013081E7
:1022A0002181F280558152955F7083819481892BC1
:1022B00039F02F3F41F481E090E03F3F31F003C01F
:1022C00081E090E002C080E090E080FD73C339833C
:1022D0002A8389819A815E830E94D919B92E8F83BE
:1022E0000E94D8190E9400192B2D22952F7030E0E2
:1022F0005E816F812530310509F4E6C06CF424302D
:1023000031050CF0A2C04B2D407F8B2D8F702230F9
:1023100031050CF045C017C02C3031054CF42A3083
:1023200031050CF0E7C12830310509F043C3E5C0A1
:102330002D30310509F4BAC20CF4A2C22F30310598
:1023400009F038C323C3182F411101C002C01295F0
:10235000107FFF2059F0112309F46BC2812F6F8386
:102360000E946F1A0E94981A6F8163C2862F0E9482
:10237000D510112309F41EC3812F0E94751A2796C8
:102380000FB6F894DEBF0FBECDBFDF91CF911F9186
:102390000F91FF90EF90DF90CF90BF900C94981A20
:1023A000403211F08295807F662319F0613071F51B
:1023B00023C0FF20B1F0511101C032C0513081F56E
:1023C00027960FB6F894DEBF0FBECDBFDF91CF9139
:1023D0001F910F91FF90EF90DF90CF90BF900C94E2
:1023E0007F1A511101C003C0513009F4E3C28E833A
:1023F0000E94821A8E819AC1FF2021F0563008F087
:10240000D9C20EC0553008F0D5C290C1FF20C9F026
:10241000552331F0F801958190FF0BC29F70958391
:1024200027960FB6F894DEBF0FBECDBFDF91CF91D8
:102430001F910F91FF90EF90DF90CF90BF900C9481
:102440002611552309F472C109C22B2D2695269514
:10245000237030E02115310529F02130310509F0D4
:10246000A9C219C0FF2021F0862F9B2D937002C0B6
:1024700080E090E027960FB6F894DEBF0FBECDBF88
:10248000DF91CF911F910F91FF90EF90DF90CF9050
:10249000BF900C94F00EFF2021F0862F9B2D93709F
:1024A00002C080E090E027960FB6F894DEBF0FBE22
:1024B000CDBFDF91CF911F910F91FF90EF90DF90F3
:1024C000CF90BF900C94060F862FFF2019F00E942A
:1024D000ED1D02C00E94551E27960FB6F894DEBF70
:1024E0000FBECDBFDF91CF911F910F91FF90EF9065
:1024F000DF90CF90BF900C94DC1E8B2D837009F081
:1025000079C0F11057C2262F229526952770220FE9
:10251000220F862F8F70C82ED12CE12CF12C022E89
:1025200004C0CC0CDD1CEE1CFF1C0A94D2F764FF27
:1025300010C06FE070E080E090E004C0660F771F8D
:10254000881F991F2A95D2F7609570958095909570
:1025500003C060E070E0CB012B2D269526952370FB
:10256000422F50E042305105D9F04330510569F116
:102570006C297D298E299F294130510551F12796DB
:102580000FB6F894DEBF0FBECDBFDF91CF911F9184
:102590000F91FF90EF90DF90CF90BF900C941519A2
:1025A0006C297D298E299F2927960FB6F894DEBFC6
:1025B0000FBECDBFDF91CF911F910F91FF90EF9094
:1025C000DF90CF90BF900C9427190E941519C70176
:1025D000B60127960FB6F894DEBF0FBECDBFDF91D0
:1025E000CF911F910F91FF90EF90DF90CF90BF9010
:1025F0000C940319FF2019F08B2D817001C0869572
:10260000882309F4D7C1262F229526952770220FFB
:10261000220F862F8F70C82ED12CE12CF12C022E88
:1026200004C0CC0CDD1CEE1CFF1C0A94D2F764FF26
:1026300010C06FE070E080E090E004C0660F771F8C
:10264000881F991F2A95D2F760957095809590956F
:1026500003C060E070E0CB012B2D269526952370FA
:10266000422F50E042305105D9F04330510569F115
:102670006C297D298E299F294130510551F12796DA
:102680000FB6F894DEBF0FBECDBFDF91CF911F9183
:102690000F91FF90EF90DF90CF90BF900C94B41902
:1026A0006C297D298E299F2927960FB6F894DEBFC5
:1026B0000FBECDBFDF91CF911F910F91FF90EF9093
:1026C000DF90CF90BF900C94C6190E94B419C70137
:1026D000B60127960FB6F894DEBF0FBECDBFDF91CF
:1026E000CF911F910F91FF90EF90DF90CF90BF900F
:1026F0000C94A219603F59F120F4603E08F494C094
:1027000008C0623F09F467C0F0F1633F09F08CC074
:1027100065C0162F1F708B2D8F71FF2021F00E9436
:102720004D19812F7DCE0E946819812F27960FB6F3
:10273000F894DEBF0FBECDBFDF91CF911F910F91F7
:10274000FF90EF90DF90CF90BF900C942D11FF2061
:10275000B1F0553008F02EC18B2D8F7127960FB632
:10276000F894DEBF0FBECDBFDF91CF911F910F91C7
:10277000FF90EF90DF90CF90BF900C948719563068
:1027800008F018C1E9CFFF2099F08B2D8F712796A3
:102790000FB6F894DEBF0FBECDBFDF91CF911F9172
:1027A0000F91FF90EF90DF90CF90BF900C944D1958
:1027B0008B2D8F7127960FB6F894DEBF0FBECDBF5D
:1027C000DF91CF911F910F91FF90EF90DF90CF900D
:1027D000BF900C946819F110EBCFD7CFFF2099F080
:1027E0008B2D8F7127960FB6F894DEBF0FBECDBF2D
:1027F000DF91CF911F910F91FF90EF90DF90CF90DD
:10280000BF900C943E1927960FB6F894DEBF0FBE0A
:10281000CDBFDF91CF911F910F91FF90EF90DF908F
:10282000CF90BF900C943919FF20A9F0552309F4DB
:10283000ACCF862F27960FB6F894DEBF0FBECDBF64
:10284000DF91CF911F910F91FF90EF90DF90CF908C
:10285000BF900C940D10552309F4AACF862F27960C
:102860000FB6F894DEBF0FBECDBFDF91CF911F91A1
:102870000F91FF90EF90DF90CF90BF900C94D51008
:102880004B2D4F70C8010E94760227960FB6F89420
:10289000DEBF0FBECDBFDF91CF911F910F91FF9093
:1028A000EF90DF90CF90BF900C946D18F11082C024
:1028B0009B2D9F70492F50E04230510599F144F40F
:1028C0004115510569F04130510509F073C019C037
:1028D00043305105C1F14430510509F06BC044C08B
:1028E00027960FB6F894DEBF0FBECDBFDF91CF9114
:1028F0001F910F91FF90EF90DF90CF90BF900C94BD
:10290000E02127960FB6F894DEBF0FBECDBFDF9152
:10291000CF911F910F91FF90EF90DF90CF90BF90DC
:102920000C94F72127960FB6F894DEBF0FBECDBFEB
:10293000DF91CF911F910F91FF90EF90DF90CF909B
:10294000BF900C94132227960FB6F894DEBF0FBEEB
:10295000CDBFDF91CF911F910F91FF90EF90DF904E
:10296000CF90BF900C942622862F27960FB6F8940E
:10297000DEBF0FBECDBFDF91CF911F910F91FF90B2
:10298000EF90DF90CF90BF900C944A224B2D4F7068
:10299000C80127960FB6F894DEBF0FBECDBFDF91FA
:1029A000CF911F910F91FF90EF90DF90CF90BF904C
:1029B0000C944C0327960FB6F894DEBF0FBECDBF24
:1029C000DF91CF911F910F91FF90EF90DF90CF900B
:1029D000BF9008950E947C1A0E94511A0E94981A72
:1029E0000E94881F0E94DC1E80E090E00E94F00E92
:1029F00080E090E00C94060F0E946C1A0C94EA148C
:102A00000E94D919292F22952F7030E02C303105E2
:102A10004CF42A3031056CF4225031092230310552
:102A200070F407C02C30310531F02F30310539F406
:102A300002C081E0089593FB882780F9089580E023
:102A40000895CF93DF9300D000D01F92CDB7DEB7AB
:102A50000F900F900F900F900F90DF91CF910895EE
:102A6000CF93DF9300D000D000D0CDB7DEB726964D
:102A70000FB6F894DEBF0FBECDBFDF91CF910895A2
:102A80001F93CF93DF93C091B20116E012C0D0E044
:102A90001C9FF0011D9FF00D1124EE57FE4F408149
:102AA000518162817381848195810E9430152196C4
:102AB000C7708091B301C813EACFDF91CF911F9106
:102AC000089540917C0150917D0160917E0170914B
:102AD0007F0180918001909181010C9430150F93BA
:102AE0001F93CF93DF938091810182958F7009F0BE
:102AF00069C080917E01882309F464C0A091B2016D
:102B0000D091B301B0917C01C0917D0180917F0192
:102B10009091800121E030E0BF3F11F020E030E0F3
:102B2000122FBC016095709506E04AC0009721F015
:102B3000CF3F29F4212F05C021E030E002C020E082
:102B400030E020FD3BC04A2F50E0049FF001059F7C
:102B5000F00D1124EE57FE4F2181C2132FC02081AA
:102B6000B2132CC02281211129C02381348128175E
:102B7000390718F0281B390B02C0260F371F283CD5
:102B80003105E0F4809181018F7080618093810133
:102B900086E0849FF001859FF00D1124E957FE4FD8
:102BA00080818F70806180838CE791E00E94341176
:102BB000DF91CF911F910F910C944015AF5FA770DB
:102BC000AD13B4CFDF91CF911F910F910895EF9284
:102BD000FF920F931F93CF93DF93CDB7DEB762972A
:102BE0000FB6F894DEBF0FBECDBF8C0185E0F801B3
:102BF000DE011D9601900D928A95E1F7D8014C9166
:102C000011965C91119712966C9112971396ED9014
:102C1000FC90149770917C01E0917D0180917F017F
:102C200090918001009739F0EF3F41F421E030E0CE
:102C30007F3F31F003C021E030E002C020E030E00F
:102C400020FD5CC120917E01222309F4F1C0E81629
:102C5000F90628F09701281B390BC90104C080959B
:102C600090958E0D9F1D883C910508F098C080912D
:102C70008101982F907F09F064C0E51314C074138C
:102C800012C0611110C08F708061809381010E9419
:102C900061158CE791E00E94341180918101D80187
:102CA00015968C9343C1EF2839F05F3F41F481E0E2
:102CB00090E04F3F31F003C081E090E002C080E03F
:102CC00090E080FD03C081E0862702C080E090E0B4
:102CD00080FF2EC08091B2012091B30136E013C075
:102CE00090E0389FF001399FF00D1124EE57FE4F10
:102CF0007181571306C07081471303C07281671337
:102D000017C0019687708213EBCF12C19F7059F0E4
:102D1000882309F40BC107C09F7029F0F801958141
:102D2000907F09F403C1805E883008F4FFC0D2C0F0
:102D3000662309F4FBC08091810181608093810149
:102D4000F5C0E51308C0741306C0611104C0D801B2
:102D500015968C939DC04D875E878D859E856A8B69
:102D60000E9400156A89882309F4B4C0662309F417
:102D7000B1C020918101822F82958F7090E00297DF
:102D80000CF4C6C080917C0190917D0198878F835F
:102D90001986FB86EA862C87CE01079646C080916D
:102DA0008101982F907F59F47E2DF98AE88A8989CC
:102DB0000E9421158CE791E00E94341195C0E51323
:102DC00011C074130FC061110DC0F8018583C801D3
:102DD0000E943411ECE7F1E086E0DF011D928A9554
:102DE000E9F7A2C04D875E878D859E856A8B0E941C
:102DF00000156A89882309F46DC0662309F46AC046
:102E000020918101822F82958F7090E002970CF4BF
:102E10007FC080917C0190917D019A8389831B8280
:102E2000FD82EC822E83CE0101960E94341170C087
:102E3000E816F90628F09701281B390BC90104C0D0
:102E4000809590958E0D9F1D883C910508F046C099
:102E5000662309F43FC0E51330C074132EC02091DF
:102E6000810120FD21C0322F32953F70832F90E0E9
:102E70000097D1F0D80115962C9315970F9741F034
:102E8000832F8F5F8295807F2F70282B15962C9330
:102E9000C8010E94341186E0F801ACE7B1E001906E
:102EA0000D928A95E1F73EC086E0F801ACE7B1E00B
:102EB00001900D928A95E1F737C04D875E878D8529
:102EC0009E850E940015811123C08091810181603F
:102ED00080938101C8010E94341126C07E2DF98A99
:102EE000E88A89890E942115ECE7F1E086E0DF019C
:102EF0001D928A95E9F70E94611518C0662351F367
:102F00004D875E878D859E850E940015882311F36D
:102F100086E0F801ACE7B1E001900D928A95E1F707
:102F20000E946F150E94611581E014C080E012C0FC
:102F30004D875E878D859E850E94D919292F229500
:102F40002F7030E0223031050CF4E0CE2430310512
:102F50000CF6E2CE62960FB6F894DEBF0FBECDBF80
:102F6000DF91CF911F910F91FF90EF9008951F93E4
:102F7000CF93DF93CDB7DEB72C970FB6F894DEBFB3
:102F80000FBECDBF4F83588769877A878B879C8711
:102F9000CE0107960E94E7158823D9F02F81388546
:102FA0008A859B85892B39F03F3F19F080E090E0BE
:102FB00004C02F3FD9F781E090E0892B09F06DC064
:102FC0004F81588569857A858B859C850E9430154F
:102FD00064C086E0FE013796DE01119601900D92E5
:102FE0008A95E1F7FF81E8854A855B8541155105A2
:102FF00039F0EF3F41F481E090E0FF3F31F003C052
:1030000081E090E002C080E090E080FD46C0209129
:10301000B30130E0C9010196877099276091B20130
:1030200070E08617970709F440C0F983EA835D834F
:103030004C8396E0929FD001939FB00D1124AE5720
:10304000BE4FFE01319601900D929A95E1F7809363
:10305000B3010E94401521C0189FC00111248E5752
:103060009E4F0E94E715882371F1E091B2011E9FE7
:10307000F0011124EE57FE4F40815181628173812E
:10308000848195810E9430158091B20190E0019673
:10309000877099278093B20101C016E08091B20138
:1030A0009091B3018913D8CF0EC00E94FC141092E6
:1030B000B3011092B201ECE7F1E086E0DF011D926E
:1030C0008A95E9F7EACF2C960FB6F894DEBF0FBECB
:1030D000CDBFDF91CF911F910895DF92EF92FF92C4
:1030E0000F931F93CF93DF93EC01009709F46CC00B
:1030F000D12CEE24E394F12C8E010F5F1F4FFE01C3
:103100008491843748F4843008F04AC0813071F0EB
:10311000823009F059C01EC0853709F43DC070F1F6
:10312000982F9458903708F04FC03DC02296F80170
:103130008491982F905E983050F48770FE2D01C0D6
:10314000FF0F8A95EAF78F2F0E946F1A30C00E94F6
:103150000D102DC02296F8018491982F905E983022
:1031600050F48770FE2D01C0FF0F8A95EAF78F2F6C
:103170000E94751A1CC00E94D51019C02296F80131
:10318000049107C08FE99FE00197F1F700C00000AC
:1031900001500111F7CF0BC02296F801D49007C05F
:1031A0000E940D1003C08F770E94D510E8018D2D6D
:1031B00007C08150EFE9FFE03197F1F700C0000050
:1031C000882309F499CFF5CFDF91CF911F910F910B
:1031D000FF90EF90DF9008956093B8017093B9016C
:1031E0008093BA019093BB010C94EA146093B401EC
:1031F0007093B5018093B6019093B7010C94EA14D3
:1032000008950C94EC180F931F930091B80110913E
:10321000B9012091BA013091BB01602B712B822B37
:10322000932B1F910F910C94EC180F931F93009107
:10323000B8011091B9012091BA013091BB0160230E
:103240007123822393231F910F910C94EC180F93F9
:103250001F930091B8011091B9012091BA013091EA
:10326000BB0160277127822793271F910F910C9430
:10327000EC1860E070E0CB010C94F61841E050E0EF
:1032800060E070E004C0440F551F661F771F8A95E9
:10329000D2F7CB01BA010C94F61841E050E060E09F
:1032A00070E004C0440F551F661F771F8A95D2F740
:1032B0008091B4019091B501A091B601B091B70190
:1032C000482B592B6A2B7B2BCB01BA010C94F61897
:1032D00041E050E060E070E004C0440F551F661FFD
:1032E000771F8A95D2F7409550956095709580919B
:1032F000B4019091B501A091B601B091B7014823F6
:1033000059236A237B23CB01BA010C94F61841E0C0
:1033100050E060E070E004C0440F551F661F771F47
:103320008A95D2F78091B4019091B501A091B60130
:10333000B091B701482759276A277B27CB01BA01EB
:103340000C94F6180F931F930091B4011091B501DE
:103350002091B6013091B701602B712B822B932BFA
:103360001F910F910C94F6180F931F930091B401C5
:103370001091B5012091B6013091B70160237123FE
:10338000822393231F910F910C94F6180F931F9390
:103390000091B4011091B5012091B6013091B701AF
:1033A00060277127822793271F910F910C94F6189D
:1033B0000895CF92DF92EF92FF920F931F93CF93D6
:1033C000DF93EC01C090B801D090B901E090BA0150
:1033D000F090BB018091B4019091B501A091B6012C
:1033E000B091B701C82AD92AEA2AFB2A0FE110E0D6
:1033F000B701A601002E04C07695679557954795AD
:103400000A94D2F740FF08C0BE01802F0E947203C9
:103410008130910509F007C00150110948F7BE013C
:1034200080E00E947203DF91CF911F910F91FF9076
:10343000EF90DF90CF90089540910C0150910D01D5
:1034400020E030E09FEFFA01E20FF31F628168177E
:10345000A1F09F3F19F4611101C0922F2F5F3F4FE0
:103460002630310581F707C0FA01E90FF11D97FDFC
:10347000FA95828308959F3FB9F7089540910C0112
:1034800050910D0120E030E0FA01E20FF31F92812C
:10349000981301C012822F5F3F4F26303105A1F7EC
:1034A000089581E090E0E0910C01F0910D01E80FAA
:1034B000F91F1082019688309105A9F7089590911F
:1034C000BC01982B9093BC01089580959091BC010C
:1034D00098239093BC0108951092BC010895909197
:1034E000BD01982B9093BD01089580959091BD01E9
:1034F00098239093BD0108951092BD010895809383
:10350000BE0108951092BE01089540910C015091A2
:103510000D0120E030E080E0FA01E20FF31F91811D
:1035200091118F5F2F5F3F4F27303105A9F7089525
:10353000E0910C01F0910D018091BC018083E0913C
:103540000C01F0910D0180819091BD01892B808348
:103550009091BE01992361F0E0910C01F0910D0171
:103560008081892B80830E94851A81110E94821A92
:1035700080910C0190910D010C94DA0E8091E00184
:10358000843009F11092C80120E488E190E00FB680
:10359000F894A895809360000FBE2093600083B7D5
:1035A000817F846083BF83B7816083BF789488956F
:1035B00083B78E7F83BF88E10FB6F8948093600055
:1035C000109260000FBE0895CF930E9474020E9473
:1035D0000E060E947502C0E08C2F0E945407892BB2
:1035E00029F4CF5FC430C1F780E001C081E0CF9102
:1035F00008950E94FC140C94CF211F920F920FB6D5
:103600000F9211248F939F93AF93BF938091C80122
:10361000811113C08091C9019091CA01A091CB0181
:10362000B091CC014196A11DB11D8093C901909329
:10363000CA01A093CB01B093CC01BF91AF919F91F0
:103640008F910F900FBE0F901F90189582E084BD50
:1036500093E095BD9AEF97BD80936E0008958FB764
:10366000F8944091C9015091CA016091CB017091C9
:10367000CC018FBFCA010895CF92DF92EF92FF92E3
:103680000F931F932FB7F8944091C9015091CA012D
:103690006091CB017091CC012FBF6A017B01EE24B8
:1036A000FF248C0120E030E0C016D106E206F306CC
:1036B00020F09A01281B390B05C09C0120953095FC
:1036C000240F351FC9011F910F91FF90EF90DF90DC
:1036D000CF9008951F920F920FB60F9211248F93DF
:1036E0009F93AF93BF938091C9019091CA01A0911C
:1036F000CB01B091CC010196A11DB11D8093C901F0
:103700009093CA01A093CB01B093CC01BF91AF912C
:103710009F918F910F900FBE0F901F9018950E9450
:10372000AD0BF8942FEF87EA91E62150804090404E
:10373000E1F700C0000087E090EBDC018093EA0134
:103740009093EB01A093EC01B093ED012CE088E1A4
:1037500090E00FB6F894A895809360000FBE209378
:103760006000FFCFCF92DF92EF92FF920F931F93F3
:10377000CF93DF93C82ED12C01E010E08D2D0E9455
:1037800054077C01C0E0D0E098010C2E02C0220F4B
:10379000331F0A94E2F72E213F21232B29F421968F
:1037A000CC30D10589F708C06C2F7D2D80E00E94B8
:1037B0004D03C812F4CF06C0D39484E0D812DECFF4
:1037C00080E001C081E0DF91CF911F910F91FF90C8
:1037D000EF90DF90CF900895CF93C82F8CE20E9496
:1037E000B21B882321F08C2FCF910C94B21B80E068
:1037F000CF910895CF930E943D1D811102C00E9478
:103800001E1DC5E608C00E940E068FE39CE90197C5
:10381000F1F700C00000C150B1F789E20E94EC1B33
:1038200081110AC18AE20E94EC1B81110E941E1DB7
:1038300085E00E94EC1B81110E948F1B0E94481D95
:103840008093C70187E00E94EC1B882399F18BE1EC
:103850000E94EC1B882351F09091C70191FB8827AF
:1038600080F921E0822780FB91F922C08EE00E943E
:10387000EC1B882351F09091C70192FB882780F9B7
:1038800021E0822780FB92F913C080E10E94EC1BAB
:103890009091C701882341F093FB882780F921E0AC
:1038A000822780FB93F904C0892F809580FB90F9D3
:1038B0009093C7018091C7010E944C1D0E945A1D20
:1038C0008093DA0180EE0E94EC1B882341F0809106
:1038D000DA01982F909590FB80F98093DA0189E3C3
:1038E0000E94EC1B882359F09091DA0191FB882704
:1038F00080F921E0822780FB91F99093DA0182EE32
:103900000E94EC1B882359F09091DA0192FB8827E2
:1039100080F921E0822780FB92F99093DA0186EE0C
:103920000E94EC1B882359F09091DA0193FB8827C1
:1039300080F921E0822780FB93F99093DA0183EEEE
:103940000E94EC1B882359F09091DA0194FB8827A0
:1039500080F921E0822780FB94F99093DA0185E3D6
:103960000E94EC1B882359F09091DA0195FB88277F
:1039700080F921E0822780FB95F99093DA0181E3B9
:103980000E94EC1B882359F09091DA0196FB88275E
:1039900080F921E0822780FB96F99093DA0181E19A
:1039A0000E94EC1B882359F09091DA0197FB88273D
:1039B00080F921E0822780FB97F99093DA018091CA
:1039C000DA010E945E1D87E20E94EC1BC82F8EE187
:1039D0000E94EC1B8111C2608FE10E94EC1B8111DF
:1039E000C46080E20E94EC1B8111C86081E20E94E9
:1039F000EC1B8111C06182E20E94EC1B8111C0624C
:103A000083E20E94EC1B8111C06484E20E94EC1BE3
:103A1000882311F0C06802C0CC2329F08C2F0E94AB
:103A2000551D6C2F03C00E94511D682F70E080E06F
:103A300090E0CF910C940119CF9108956DEE7EEF37
:103A400080E090E00E94CC2360E082E090E00E9461
:103A5000BE2360E083E090E00E94BE2360E084E04B
:103A600090E00E94BE2360E085E090E00E94BE23CB
:103A700060E086E090E00C94BE2380E090E00E943D
:103A8000B82321E08D3E9E4F09F020E0822F08955B
:103A900082E090E00C94B023682F82E090E00C94D8
:103AA000BE2383E090E00C94B023682F83E090E085
:103AB0000C94BE2384E090E00C94B023682F84E043
:103AC00090E00C94BE2386E090E00C94B023682F25
:103AD00086E090E00C94BE238091D50180FF0BC05E
:103AE0006091110185E0689FB0011124759567957B
:103AF000759567952AC081FF09C06091110185E025
:103B0000689FB0011124759567951FC082FF07C09B
:103B10006091110185E0689FB001112416C04091A9
:103B2000CF014423C9F060911001461788F7209116
:103B3000110185E0289F90011124429FC001439FFD
:103B4000900D112470E00E9488236038710540F4C4
:103B50006115710539F002C065E070E0862F0895A7
:103B60008FE7089581E008958091D50180FF08C016
:103B700060910F0170E0759567957595679521C007
:103B800081FF06C060910F0170E07595679519C0BF
:103B900082FF04C060910F0170E010C08091CF01DE
:103BA0008823C1F060910E018617A0F790910F0154
:103BB000989FC001112470E00E948823603871052D
:103BC00028F46115710521F0862F08958FE7089577
:103BD00081E0089561E070E0F4CF803F21F40E941D
:103BE0006C1D819504C0813F29F40E946C1D809357
:103BF000D2010895823F21F40E946C1D819504C07A
:103C0000833F29F40E946C1D8093D1010895893F60
:103C100019F40E94B41D05C08A3F31F40E94B41DFE
:103C200081958093D30108958B3F21F40E94B41DA8
:103C3000819504C08C3F29F40E94B41D8093D40167
:103C40000895843F21F48091D001816017C0853FA1
:103C500021F48091D001826011C0863F21F48091CF
:103C6000D00184600BC0873F21F48091D00188602F
:103C700005C0883F31F48091D00180618093D001EC
:103C800008958D3F21F48091D50181600BC08E3F56
:103C900021F48091D501826005C08F3F29F4809185
:103CA000D50184608093D5010895803F29F48091E7
:103CB000D20187FF6EC007C0813F41F48091D201DD
:103CC00018160CF066C01092D20163C09091D10119
:103CD000823F19F497FF5DC005C0833F31F4191688
:103CE0000CF057C01092D10154C0893F31F480913B
:103CF000D30118160CF04DC006C08A3F39F48091EC
:103D0000D30187FF46C01092D30143C08B3F29F4F3
:103D10008091D40187FF3DC006C08C3F39F480916B
:103D2000D4011816B4F51092D40133C0843F21F4A5
:103D30008091D0018E7F05C0853F31F48091D00104
:103D40008D7F8093D00125C0863F21F48091D001E2
:103D50008B7FF7CF873F21F48091D001877FF1CF10
:103D6000883F21F48091D0018F7EEBCF8D3F21F4ED
:103D70008091D5018E7F0BC08E3F21F48091D501BB
:103D80008D7F05C08F3F29F48091D5018B7F809373
:103D9000D5018091D10181110EC08091D201811194
:103DA0000AC08091D301811106C08091D401811194
:103DB00002C01092CF01089580ED91E00E94E50EBF
:103DC0000E942F1B9093CE018093CD010895CF9335
:103DD0008091CD019091CE010E943C1B4091CF017A
:103DE000442321F02091120130E006C020911301FC
:103DF0005AE0259F900111248217930708F486C08A
:103E00008091D10181110DC09091D201911109C011
:103E10009091D301911105C09091D401992309F497
:103E200075C04F3F19F04F5F4093CF01181624F42F
:103E30000E946C1D8093D1018091D10187FF05C044
:103E40000E946C1D81958093D1018091D20118163A
:103E500024F40E946C1D8093D2018091D20187FFCF
:103E600005C00E946C1D81958093D2016091D101A3
:103E7000662339F1C091D201CC2319F1772767FD70
:103E80007095872F972F0E94992223E333E343E312
:103E90005FE30E94FD220E9466226093D1016C2F95
:103EA000772767FD7095872F972F0E94992223E32C
:103EB00033E343E35FE30E94FD220E9466226093A6
:103EC000D2018091D301181624F40E94B41D80936E
:103ED000D3018091D30187FF05C00E94B41D819555
:103EE0008093D3018091D401181624F40E94B41D4C
:103EF0008093D4018091D40187FF05C00E94B41D36
:103F000081958093D401CF910C94DC1ECF910895BC
:103F1000E0EDF1E085E0DF011D928A95E9F710926E
:103F2000CF011092D5010895833089F130F48130AA
:103F300061F0823009F06EC019C0853009F449C0C3
:103F4000B8F1863009F066C055C020911301862F64
:103F500090E0820F911D8F3F910520F4620F6093D6
:103F6000130108958FEF809313010895209112019A
:103F7000862F90E0820F911D8F3F910520F4620FF4
:103F80006093120108958FEF80931201089520919C
:103F90001101862F90E0820F911D8F3F910520F433
:103FA000620F6093110108958FEF809311010895BE
:103FB00020911001862F90E0820F911D8F3F910577
:103FC00020F4620F6093100108958FEF8093100129
:103FD000089520910F01862F90E0820F911D8F3F51
:103FE000910520F4620F60930F0108958FEF809385
:103FF0000F01089520910E01862F90E0820F911DF0
:104000008F3F910520F4620F60930E0108958FEFAA
:1040100080930E010895833021F130F4813059F0FE
:10402000823009F049C012C0853089F128F186300C
:1040300009F042C037C080911301681720F4861B35
:104040008093130108951092130108958091120135
:10405000681720F4861B80931201089510921201B4
:10406000089580911101681720F4861B8093110137
:10407000089510921101089580911001681720F49D
:10408000861B80931001089510921001089580916D
:104090000F01681720F4861B80930F01089510927A
:1040A0000F01089580910E01681720F4861B8093FC
:1040B0000E01089510920E01089541E050E060E075
:1040C00070E004C0440F551F661F771F8A95D2F712
:1040D000CB01BA010E9401190C94FC14873208F537
:1040E0008E3108F0B9C08E3009F47EC060F487309C
:1040F00009F465C018F4863059F549C0883051F18B
:104100008B3031F5AEC0883130F4863108F0A9C06B
:104110008031F1F473C0893109F4A3C08B31C1F44B
:1041200059C08933F1F068F4893209F493C018F466
:10413000873271F48FC0853309F48CC0883341F421
:1041400090C0863409F46BC008F488C0883449F103
:1041500080E008950E94481D0E945A1D0E94631D20
:1041600080C00E94C90E892B59F00E94C90E9093FD
:10417000D8018093D7010E94FC1480E090E004C035
:104180008091D7019091D8010E94C40E6AC080919D
:10419000C701817F8E7F8093C70181E08093D60124
:1041A00008950E94FC142FEF83ED90E3215080408E
:1041B0009040E1F700C000000E948F1B52C0809128
:1041C000C70180FF03C0817F8E7F01C08160809323
:1041D000C70147C09091C70191FB882780F921E072
:1041E000822780FB91F913C09091C70192FB882729
:1041F00080F921E0822780FB92F909C09091C701E4
:1042000093FB882780F921E0822780FB93F9909324
:10421000C701882331F191609093C70122C081E8E2
:1042200090E00E94F00E2FEF81EE94E0215080404C
:104230009040E1F700C0000080E090E00E94F00EA6
:104240002FEF89E698E1215080409040E1F700C0CF
:10425000000007C080E003C08D5101C089530E9457
:104260005D2081E0089580E0089580E00895CF9377
:10427000C82F8091D601813071F020F0823009F092
:1042800083C037C0A0910C01B0910D018C91823296
:1042900009F07CC007C0A0910C01B0910D018C9178
:1042A000823249F48C2F0E94332181111EC08C2F41
:1042B0000E946E201CC08C2F0E943521811115C0D8
:1042C000C43169F030F4CB3081F0C03109F062C004
:1042D00009C0C93221F0C83309F05CC006C0109291
:1042E000D60158C082E08093D60181E090E08170D1
:1042F00054C0C932C1F060F4C431A9F020F4C73011
:1043000009F046C02EC0CE51CA3008F041C011C0DD
:10431000CE3409F118F4CB34D9F517C0C13599F072
:10432000C235B1F50EC01092D90181E08093D6015B
:1043300034C0EC2FF0E0E85BFE4F80818093D90120
:1043400027C061E003C061E007C06AE08091D90145
:104350000E94941F1DC06AE08091D9010E940B2029
:1043600017C08EE18093130182E3809312018AE0EB
:104370008093110184E18093100188E080930F0104
:1043800088E280930E0104C01092D60180E005C03F
:1043900081E003C080E090E0AACFCF9108950E9411
:1043A0003D1D811102C00E941E1D0E94631D80934D
:1043B000E90180FF02C0869501C080E00C945F0790
:1043C0008091E901982F9695292F30E0233031050F
:1043D0004CF49F5F990F8170892B81608093E90174
:1043E0000E94671D8091E90186950C945F0780917A
:1043F000E901982F969591F09158990F8170892B2A
:104400008093E9018E7F91E009F490E08091E901C9
:1044100090FB80F98093E9010E94671D8091E9017A
:1044200086950C945F078091E901982F909590FBF9
:1044300080F98093E9010E94671D8091E90180FF66
:1044400002C0869501C080E00C945F073091E901BD
:10445000232F26952F5F2F77822F90E031700497BE
:104460002CF4220F232B2093E90102C03093E901A1
:104470008091E901282F2E7F91E009F490E090FBD4
:1044800080F98093E9010E94671D8091E90186957A
:104490000C945F072091E901922F96959827990F28
:1044A000822F8170892B8093E9018E7F91E009F43E
:1044B00090E08091E90190FB80F98093E9010E94EE
:1044C000671D8091E90186950C945F0704D068947C
:1044D000B1118DC0089570D088F09F5790F0B92F1A
:1044E0009927B751A0F0D1F0660F771F881F991F49
:1044F0001AF0BA95C9F712C0B13081F077D0B1E0A7
:10450000089574C0672F782F8827B85F39F0B93FB6
:10451000CCF3869577956795B395D9F73EF490954A
:104520008095709561957F4F8F4F9F4F0895E894C8
:1045300009C097FB3EF490958095709561957F4FEB
:104540008F4F9F4F9923A9F0F92F96E9BB27939599
:10455000F695879577956795B795F111F8CFFAF4A9
:10456000BB0F11F460FF1BC06F5F7F4F8F4F9F4FDA
:1045700016C0882311F096E911C0772321F09EE838
:10458000872F762F05C0662371F096E8862F70E09E
:1045900060E02AF09A95660F771F881FDAF7880F78
:1045A0009695879597F9089557FD9058440F551F94
:1045B00059F05F3F71F04795880F97FB991F61F0A5
:1045C0009F3F79F087950895121613061406551F1C
:1045D000F2CF4695F1DF08C0161617061806991F88
:1045E000F1CF86957105610508940895E894BB277D
:1045F00066277727CB0197F908950BD078C069D04B
:1046000028F06ED018F0952309F05AC05FC011242D
:10461000EECFCADFA0F3959FD1F3950F50E0551F61
:10462000629FF001729FBB27F00DB11D639FAA2707
:10463000F00DB11DAA1F649F6627B00DA11D661F56
:10464000829F2227B00DA11D621F739FB00DA11D77
:10465000621F839FA00D611D221F749F3327A00D31
:10466000611D231F849F600D211D822F762F6A2FCD
:1046700011249F5750408AF0E1F088234AF0EE0F52
:10468000FF1FBB1F661F771F881F91505040A9F75F
:104690009E3F510570F014C0AACF5F3FECF3983EE7
:1046A000DCF3869577956795B795F795E7959F5FC6
:1046B000C1F7FE2B880F911D9695879597F9089560
:1046C00097F99F6780E870E060E008959FEF80ECC5
:1046D000089500240A941616170618060906089568
:1046E00000240A9412161306140605060895092ECE
:1046F0000394000C11F4882352F0BB0F40F4BF2B3D
:1047000011F460FF04C06F5F7F4F8F4F9F4F08957C
:1047100097FB072E16F4009407D077FD09D00E946E
:104720009C2307FC05D03EF4909581959F4F0895FA
:10473000709561957F4F0895AA1BBB1B51E107C07F
:10474000AA1FBB1FA617B70710F0A61BB70B881F21
:10475000991F5A95A9F780959095BC01CD010895B0
:10476000F999FECF92BD81BDF89A992780B5089539
:10477000A8E1B0E042E050E00C94D323262FF99951
:10478000FECF1FBA92BD81BD20BD0FB6F894FA9A34
:10479000F99A0FBE019608950E94BE23272F0C940C
:1047A000BF23DC01CB01FC01F999FECF06C0F2BDAD
:1047B000E1BDF89A319600B40D9241505040B8F7DF
:0647C0000895F894FFCFFC
:1047C600058E071E08FA07C507910701BF012808CD
:1047D600140A321E400045002500260061006000D4
:1047E600200037006400650066006700440046004C
:1047F6002400470006031F03380351031D04D0039A
:104806009A037A033F4D3620010203040506070882
:02481600090097
:00000001FF
